:100000000C9434000C9451000C9451000C94510049
:100010000C9451000C9451000C9451000C94FC0071
:100020000C9451000C9451000C9451000C94CB0092
:100030000C9451000C9451000C949A000C945100B3
:100040000C9451000C9451000C9451000C945100EC
:100050000C9451000C9451000C9451000C945100DC
:100060000C9451000C94510011241FBECFEFD8E026
:10007000DEBFCDBF11E0A0E0B1E0ECEAF5E002C0E8
:1000800005900D92A631B107D9F711E0A6E1B1E0D4
:1000900001C01D92AB31B107E1F70E944F010C94F2
:1000A000D4020C940000FC01A685B7858C91829542
:1000B000817080871186848995898230910561F0ED
:1000C0008330910599F00197C9F416BC80916E00B8
:1000D000826080936E0016C010928500109284009A
:1000E00080916F00826080936F000CC01092B2000C
:1000F0008091700082608093700004C081E090E085
:100100000E94D40278949FB7F894809118019FBF01
:100110008823C9F310921801A089B189808591853F
:10012000009721F08C9182608C9308958C918D7F43
:100130008C9308951F920F920FB60F9211242F9354
:100140003F938F939F938091160190911701019691
:10015000909317018093160180911801813091F0DE
:1001600020911601309117018091190190911A0187
:100170002817390738F081E0809318011092170191
:10018000109216019F918F913F912F910F900FBE6A
:100190000F901F9018951F920F920FB60F92112477
:1001A0002F933F938F939F93809116019091170106
:1001B0000196909317018093160180911801813068
:1001C00091F02091160130911701809119019091C1
:1001D0001A012817390738F081E08093180110922E
:1001E0001701109216019F918F913F912F910F90BF
:1001F0000FBE0F901F9018951F920F920FB60F927F
:1002000011242F933F938F939F9380911601909188
:1002100017010196909317018093160180911801A0
:10022000813091F0209116013091170180911901D0
:1002300090911A012817390738F081E0809318014E
:1002400010921701109216019F918F913F912F915B
:100250000F900FBE0F901F901895FC01219A85E218
:1002600090E0918B808B249883E290E0978786873B
:1002700085B5836085BD81E090E0938B828B22E021
:1002800030E030931A012093190124B5226024BD77
:1002900029EF27BD958B848B80E090E00895CF9265
:1002A000DF92EF92FF9280E091E00E942D01C12C3D
:1002B000D12C760160E070E0CB0160930001709377
:1002C0000101809302019093030180E091E00E947C
:1002D00053008FEFC81AD80AE80AF80AC701B60116
:1002E0000E94E3012FE632E143E05BE30E947102EA
:1002F00020E030E0A9010E947F01DFCF5058BB27EA
:10030000AA270ED0B4C0A5D030F0AAD020F031F486
:100310009F3F11F41EF49AC00EF4E095E7FB90C0E5
:10032000E92FB6D080F3BA176207730784079507E1
:1003300018F071F49EF5CEC00EF4E0950B2EBA2F96
:10034000A02D0B01B90190010C01CA01A0011124DB
:10035000FF27591B99F0593F50F4503E68F11A1687
:10036000F040A22F232F342F4427585FF3CF469518
:1003700037952795A795F0405395C9F77EF41F163A
:10038000BA0B620B730B840BBAF09150A1F0FF0F04
:10039000BB1F661F771F881FC2F70EC0BA0F621FF0
:1003A000731F841F48F4879577956795B795F795E0
:1003B0009E3F08F0B3CF9395880F08F09927EE0F72
:1003C000979587950895E89409C097FB3EF490951A
:1003D0008095709561957F4F8F4F9F4F9923A9F01E
:1003E000F92F96E9BB279395F695879577956795AD
:1003F000B795F111F8CFFAF4BB0F11F460FF1BC0F1
:100400006F5F7F4F8F4F9F4F16C0882311F096E983
:1004100011C0772321F09EE8872F762F05C0662331
:1004200071F096E8862F70E060E02AF09A95660FEA
:10043000771F881FDAF7880F9695879597F90895A3
:1004400097F99F6780E870E060E008959FEF80EC87
:10045000089500240A94161617061806090608952A
:1004600000240A9412161306140605060895092E90
:100470000394000C11F4882352F0BB0F40F4BF2BFF
:1004800011F460FF04C06F5F7F4F8F4F9F4F08953F
:1004900057FD9058440F551F59F05F3F71F0479535
:1004A000880F97FB991F61F09F3F79F0879508951A
:1004B000121613061406551FF2CF4695F1DF08C039
:1004C000161617061806991FF1CF86957105610556
:1004D00008940895E894BB2766277727CB0197F9FE
:1004E00008950BD0C4CFB5DF28F0BADF18F09523FC
:1004F00009F0A6CFABCF1124EECFCADFA0F3959FB2
:10050000D1F3950F50E0551F629FF001729FBB27FA
:10051000F00DB11D639FAA27F00DB11DAA1F649FA6
:100520006627B00DA11D661F829F2227B00DA11D59
:10053000621F739FB00DA11D621F839FA00D611DDF
:10054000221F749F3327A00D611D231F849F600D00
:10055000211D822F762F6A2F11249F5750408AF039
:10056000E1F088234AF0EE0FFF1FBB1F661F771FC5
:10057000881F91505040A9F79E3F510570F060CF01
:10058000AACF5F3FECF3983EDCF3869577956795AD
:10059000B795F795E7959F5FC1F7FE2B880F911DE3
:0C05A0009695879597F90895F894FFCF81
:1005AC00000000000000000000006F12033B000080
:0605BC0000000000000039
:00000001FF
